:020000040800F2
:10000000E8150020650100088D1900083514000866
:10001000891900087F020008CD2D000800000000AB
:10002000000000000000000000000000F1220008B5
:10003000BD10000800000000D11B00087D2B000847
:100040007F0100087F0100087F0100087F01000890
:100050007F0100087F0100087F0100087F01000880
:100060007F0100087F0100087F0100087F01000870
:100070007F0100087F0100087F0100087F01000860
:100080007F0100087F0100087F010008692C00083B
:10009000412D00087F0100087F0100087F01000852
:1000A0007F0100087F0100087F0100087F01000830
:1000B0007F0100087F0100087F0100087F01000820
:1000C0007F0100087F0100087F0100087F01000810
:1000D0007F0100087F0100087F0100087F01000800
:1000E0007F0100087F0100087F0100087F010008F0
:1000F0007F0100087F0100087F0100087F010008E0
:100100007F0100087F0100087F0100087F010008CF
:100110007F0100087F0100087F0100087F010008BF
:100120007F0100087F0100087F0100087F010008AF
:10013000DFF80CD000F046F80048004741400008C6
:10014000E8150020EFF30980704780F309887047B5
:10015000EFF30880704780F30888704740BA704713
:10016000C0BA70470648804706480047FEE7FEE7EA
:10017000FEE7FEE7FEE7FEE7FEE7FEE7FEE7FEE757
:10018000812B000831010008421C10F8011B0029D6
:10019000FBD1801A704730B50B4601460020202263
:1001A000012409E021FA02F59D4205D303FA02F584
:1001B000491B04FA02F52844151EA2F10102F1DCE4
:1001C00030BD0000064C074D06E0E06840F001033A
:1001D00094E8070098471034AC42F6D3FFF7ACFF21
:1001E000204600084046000870B58C1810F8015BE6
:1001F00015F0070301D110F8013B2A1106D110F8C0
:10020000012B03E010F8016B01F8016B5B1EF9D1C3
:100210002B0705D40023521E0DD401F8013BFAE749
:1002200010F8013BCB1A921C03E013F8015B01F8B4
:10023000015B521EF9D5A142D8D3002070BD10B584
:10024000044624B1012C07D0022C15D10AE010215C
:10025000012002F00FF910E04FF48051022002F06B
:10026000B1F80AE01021012002F004F94FF48051A6
:10027000022002F0A7F800E000BF00BF10BD00BFE1
:10028000FEE70146CAB20B1243EA022070470000A3
:1002900010B5002404E0A748005DA7490855641C78
:1002A000A64800888442F6D3A3484068A449486021
:1002B000A14880688860A14800881F280FD00220CC
:1002C000FFF7BDFF00209C490860487B1A220521EA
:1002D00002F094F90021012002F072F910BD964855
:1002E000C07B282803D09448C07B2A2816D1924886
:1002F000407C01069048807C41EA00418E48C07CE9
:1003000041EA00208C49097D08438E4908608A48EB
:10031000C17D807D41EA00208B49086086480068E5
:100320008A4988426FD18448407B8949096888425C
:1003300007D88148807B012803DB7F48807B102819
:100340000DDD0220FFF77BFF7B49487B242205213E
:1003500002F054F90021012002F032F9E8E0764879
:10036000C07B25285FD01BDC15286FD00EDC082849
:100370006DD006DC00285BD0032830D0042867D17C
:1003800076E00A2873D01228F9D12DE01A380A280D
:100390005ED2DFE800F0392EB17D33B1B1B1B143A7
:1003A0008A286FD00EDC552867D006DC282844D078
:1003B0002A284ED02F28E2D154E05A2829D0882864
:1003C000DDD176E0A8286DD004DC8F286FD09E2880
:1003D000D5D173E0AA287BD0AF28D0D182E056498E
:1003E000487B01F08DFE95E05349487B01F060FDAC
:1003F00090E05149487B01F097FE8BE04E49487BE5
:1004000001F092FE86E086E04B49487B01F0A0FDBA
:1004100080E04949487B01F091FD7BE04649487BFB
:1004200001F02AFE76E04449487B01F0D7FD71E0F7
:100430004149487B01F080FE6CE03F49487B4249DE
:100440000A684049096801F08DFD63E01BE024E083
:1004500052E03949487B3C490A683A49096801F049
:10046000A7FE57E03449487B01F082FE52E02AE0C3
:100470003149487B01F004FD4CE02F49487B01F0F5
:100480003BFD47E029E02C49487B01F035FD41E088
:100490002949487B01F030FD3CE02749487B01F0C9
:1004A0002BFD37E02449487B01F026FD32E01EE0B9
:1004B0000EE02149487B01F01FFD2BE01E49487BDF
:1004C00001F01AFD26E01C49487B01F015FD21E0F2
:1004D0001949487B01F010FD1CE01749487B01F0E9
:1004E0000BFD17E01449487B01F006FD12E01249AC
:1004F000487B01F001FD0DE00220FFF7A0FE0E4950
:10050000487B2022052102F079F80021012002F029
:1005100057F800BF0CE00220FFF791FE0649487B28
:100520002022052102F06AF80021012002F048F89B
:1005300000BFD3E65C1100209C110020DE020020E9
:10054000BC110020E0020020E40200205553424389
:100550004003002010B5002449E047F6FF70294908
:1005600008602948008800F00F00284908700846F4
:100570000078274901EB8000D0F8000C84B204F425
:100580000040C8B12148007801EB8000D0F8000C91
:10059000C0F30E0048F68F7108401C4909781C4AC8
:1005A00002EB8101C1F8000C18490978491E194A6B
:1005B00052F8210080471AE004F08000B8B11348D7
:1005C0000078134901EB8000D0F8000C48F60F7159
:1005D00008400E4909780E4A02EB8101C1F8000C6F
:1005E0000A490978491E0C4A52F8210080470548FB
:1005F000006880B20449088000F400400028ACD1B3
:1006000010BD0000445C004004030020E003002013
:1006100000500040240300200803002008B50020FB
:10062000009022E19748008800F00F00964908707A
:100630000846007800287CD19448006894490880D6
:100640000846008800F030009249088090480088F1
:1006500000F440508E4908808C4909684BF6BF72FF
:1006600001EA020080F4005080F0200040F40041D4
:1006700041F08001854A11608248008800F0100036
:1006800090BB1046006848F60F710840114608609C
:1006900000F0D2FE7D4909684BF6BF7201EA020004
:1006A0007B49098801F4805109B180F48050784970
:1006B000098801F4005109B180F400507549098896
:1006C00001F0100109B180F010007249098801F0B1
:1006D000200109B180F0200081B241F4004141F0D5
:1006E00080016A4A116008BDFFE76848006880B26F
:1006F0000090BDF8000000F40060B0B363480068EB
:10070000C0F30E0048F68F7108406049086001F0A0
:100710008FFF5E4909684BF6BF7201EA02005C492F
:10072000098801F4805109B180F480505849098842
:1007300000E056E001F4005109B180F40050554941
:10074000098801F0100109B180F0100051490988B1
:1007500001F0200109B180F0200081B241F4004194
:1007600041F08001494A1160BDE7FFE7BDF8000094
:1007700000F40040002878D044480068C0F30E0020
:1007800048F68F7108404149086001F0E5F93F499A
:1007900009684BF6BF7201EA02003D49098801F47D
:1007A000805109B180F480503949098801F4005121
:1007B00009B180F400503749098801F0100109B1EE
:1007C00080F010003349098801F0200109B180F060
:1007D000200081B241F4004141F080012B4A1160B8
:1007E00081E7294800782C4901EB8000D0F8000C03
:1007F00080B20090BDF8000000F40040C0B1224873
:10080000007801EB8000D0F8000CC0F30E0048F631
:100810008F7108401C4909781F4A02EB8101C1F819
:10082000000C19490978491E1C4A52F821008047DA
:10083000BDF8000000F08000B8B1134800781649F8
:1008400001EB8000D0F8000C48F60F7108400E490B
:100850000978114A02EB8101C1F8000C0A490978B4
:10086000491E0F4A52F8210080470848443000686A
:1008700080B20449088000F4004000287FF4D2AE22
:1008800000BF30E704030020E0030020005C0040CC
:10089000F4030020F6030020005000402403002051
:1008A000080300200B4A02EB8001D1F8001C01F480
:1008B000804171B102EB8001D1F8001C48F68F72C3
:1008C00011404CF280021143024B03EB8002C2F84C
:1008D000001C7047005000400B4A02EB8001D1F829
:1008E000001C01F0400171B102EB8001D1F8001C45
:1008F00048F68F72114048F2C0021143024B03EBDD
:100900008002C2F8001C704700500040084A02EB09
:100910008001D1F8001C48F68F62114048F2800235
:100920001143034B03EB8002C2F8001C7047000028
:10093000005000407FB500218F4802F0E0FE8F4953
:100940008F4803F0BCF88F48FFF71EFC8D4946180E
:100950008A48C088C0F345108849C988C90A874AAF
:100960009288520A02F2BC72844B9B88C3F34313F1
:10097000CDE90032CDE902108048007900F01F0374
:100980007F4A81A1304602F0D7FA7E48FFF7FCFB90
:100990007C494618864887A10268304602F0CCFAA6
:1009A0004FF48061744802F0AAFE884B8022884987
:1009B000714802F0BBFF8648006886490968884292
:1009C00026D07048FFF7E0FB6E49461882A13046FA
:1009D00002F0B2FA6B48FFF7D7FB6A49461885A1C7
:1009E000304602F0A9FA6748FFF7CEFB6549461882
:1009F0008CA1304602F0A0FA9148006838B14FF45B
:100A00000073604A8E480168002000F0CFFD7FBD72
:100A10005C48FFF7B9FB5B4946186D4A89A130462F
:100A200002F08AFA0021544802F069FE6049086821
:100A3000C11700EB11610912A0EB0121864A116078
:100A40005B48006811460968401A84490860002024
:100A50008349086000F0D6FB00240AE000BF00F0E4
:100A600077FB0428FBD17F4901EBC42000F030FB69
:100A7000641C4F490868C11700EB5151012202EB79
:100A8000E121A142EADC3F48FFF77EFB3D494618E1
:100A900075A1304602F050FA002421E04B4B4FF490
:100AA00080724B49344802F041FF774908700025B5
:100AB0000CE000BF00F04CFB0428FBD1444A515924
:100AC000684A2244501900F067FB2D1DFF2DF0DD10
:100AD0006348006800F580706149086004F580741F
:100AE0005E4800688442D9D3384B5B483849026875
:100AF000214802F01BFF644908700AE0564800686C
:100B0000401C55490860FF2153480068401E304A88
:100B100011545148007800F003000028EED1002461
:100B20000EE000BF00F014FB0428FBD1284A115945
:100B30004B4A12684B4B1A44101900F02DFB241D30
:100B4000454800688442ECD300F01CFB0D48FFF7D9
:100B50001BFB0C4946184DA1304602F0EDF9384810
:100B6000006838B14FF40073064A35480168002028
:100B700000F01CFD00BF4AE72806002044090020C1
:100B80004A450008200000200D0A46696C652025B2
:100B900073205B253032752E253032752E25752059
:100BA000253032753A253032755D0D0A000000009F
:100BB0000C00002046696C652073697A6520256405
:100BC0002062797465730D0A00000000080000209F
:100BD000440800206C4500084E6F742066696E64FE
:100BE000202070726F67616D6D2049442121210DB5
:100BF0000A000000436F707920636F72726563743E
:100C00002062696E6172792066696C652066726F18
:100C10006D206674702E69666163652E72750D0AAB
:100C20000000000057726974652070726F6772610E
:100C30006D2063616E63656C65642E2E2E0D0A0057
:100C40001C00002050726F6772616D6D2049443A3C
:100C5000202573200D0A0000140000201000002041
:100C60001800002000000108436C6561722070725A
:100C70006F6772616D6D206D656D6F7279202D20CB
:100C80004F4B210D0A0000000500002057726974C7
:100C9000652070726F6772616D6D20636F6D6C653A
:100CA0007465210D0A0000002DE9F047284800680E
:100CB00000F110052E8826480068077AD6B9042F5F
:100CC00018D12448007801280FD10021224800685B
:100CD00080B2801C214A42F8101030202049088040
:100CE00000BF00201B49087003E0072710201C49A3
:100CF000088027E0AC88A64201D8042000E002204A
:100D00000746B44200D93446A0B2A9688847804655
:100D1000002000F047FB8146A2B24946404602F05F
:100D200057F8A1B2002001F097FB2888001B28800B
:100D300068882044688030200949088000020949F9
:100D4000088000BF024909680F72BDE8F087000003
:100D5000E4030020DE030020505C004000600040FF
:100D6000F6030020F40300202DE9F0412848006834
:100D700000F110042688A068C0B1BEB1A588B542B4
:100D800000D93546A8B2A168884707462088401B8D
:100D90002080608828446080002000F0E1FA8046CE
:100DA000AAB24146384600F0FFFE00BF208850B18D
:100DB0004FF44050174908800021084601F04CFBD1
:100DC0003020154908802088A188884204DB032050
:100DD0000F490968087218E02088002804DD052002
:100DE0000B490968087210E0208870B9062008498C
:100DF0000968087200210948006880B2801C084A0E
:100E000042F81010302004490880BDE8F08100004D
:100E1000E4030020F4030020F6030020505C0040AF
:100E2000006000402DE9F84F9B4800684578002796
:100E3000BA46062D1BD198480068007800F07F0064
:100E4000002813D1944909688878012803D193496F
:100E50000968CF690AE0022803D1904909680F6A3E
:100E600004E0032802D18D4909684F6A94E0002DFF
:100E700064D189480068408800285FD186480068AE
:100E8000C08802285AD1844800680079002855D1CA
:100E900081480068007800F07F0028B97E4800682B
:100EA000808808B97E4F77E07B480068007800F0C2
:100EB0007F00012810D17849096848797749096885
:100EC0008A6900219047002866D173480068807ABB
:100ED000002861D0724F5FE06F480068007800F032
:100EE0007F00022858D16C480068407900F00F0656
:100EF00069480068407900F07009674800684079E7
:100F000000F0800038B1674901EB8600D0F8000C92
:100F100000F0300806E0634901EB8600D0F8000CD1
:100F200000F4405860480078B04235D9B9F1000F5C
:100F300032D1B8F1000F2FD0594F2DE0082D07D135
:100F400055480068007800F07F0028BB574F23E029
:100F50000A2D21D150480068007800F07F00012858
:100F60001AD14D480068807AB0B14B48006840887B
:100F700090B949480068007970B947480068C0884E
:100F8000012809D1444909684879444909688A69AE
:100F90000021904700B9464F57B13F480068A0F87C
:100FA00012A03D48006887610020B84700240FE088
:100FB000394A12685078394A1268116988470446DC
:100FC000032C05D10920344909680872BDE8F88F5F
:100FD00031480068008A4FF6FF71884204D1092029
:100FE0002D4909680872F1E7022C03D02A480068ED
:100FF000008A20B90820284909680872E6E72648CF
:101000000068007800F08000E0B323480068C088E2
:10101000009021480068008A0099884204D91E493E
:1010200000980968088223E01B480068008A1A4972
:101030000968C98888421BDA17480068008A17497E
:10104000096891F82C10884203DA002019490870C9
:101050000EE011480068008A1049096891F82C10C8
:1010600090FBF1F201FB120010B901201149087048
:101070000A48006890F82C10074800688182FFF742
:1010800013FE07E0FFE70320034909680872000325
:101090000949088000BF99E7E4030020E803002025
:1010A000D1280008005000404403002055280008C3
:1010B000A5280008DE030020F4030020704710B5C7
:1010C00000F0C2FB10BD10B500F0F8FB10BD000031
:1010D00030B5044604254FF4302000F09FF8054653
:1010E000042D17D10C48006940F002000A4908613C
:1010F00008464461006940F0400008614FF4302028
:1011000000F08CF805460448006941F6FD7108407E
:1011100001490861284630BD0020024004200B49E7
:10112000C96801F0010109B101200EE00749C96851
:1011300001F0040109B1022007E00449C96801F087
:10114000100109B1032000E0042070470020024094
:1011500004200B49C96801F0010109B101200EE02A
:101160000749C96801F0040109B1022007E00449F8
:10117000C96801F0100109B1032000E004207047A4
:10118000002002400348006940F0800001490861E6
:10119000704700000020024078B506460C46042542
:1011A00000200090E80200F039F80546042D24D113
:1011B0001348006940F00100114908613480E802D9
:1011C00000F02CF80546042D10D1B01C0090200C26
:1011D00000990880E80200F021F8054608480069F7
:1011E00041F6FE7108400649086106E004480069BE
:1011F00041F6FE71084002490861284678BD0000AA
:101200000020024002480349486003484860704794
:101210002301674500200240AB89EFCD00B50246AF
:101220000423FFF77BFF034603E0FFF777FF034646
:10123000521E012B01D1002AF7D102B9052318460D
:1012400000BD2DE9F04102460025002600200023C4
:101250000024002791F803C00CF00F0591F803C09B
:101260000CF0100CBCF1000F03D091F802C04CEA56
:10127000050591F800C0BCF1000F31D014680020C2
:101280002BE04FF0010C0CFA00F3B1F800C00CEAAF
:1012900003069E4220D183004FF00F0C0CFA03F797
:1012A000BC4305FA03FC4CEA040491F803C0BCF10A
:1012B000280F06D14FF0010C0CFA00FCC2F814C044
:1012C0000AE091F803C0BCF1480F05D14FF0010CC2
:1012D0000CFA00FCC2F810C0401C0828D1D31460DE
:1012E000B1F800C0BCF1FF0F34DD546800202EE0DF
:1012F00000F1080C4FF0010808FA0CF3B1F800C037
:101300000CEA03069E4221D183004FF00F0C0CFA29
:1013100003F7BC4305FA03FC4CEA040491F803C04C
:10132000BCF1280F05D100F1080C08FA0CF8C2F83E
:10133000148091F803C0BCF1480F07D100F1080CEC
:101340004FF0010808FA0CF8C2F81080401C082879
:10135000CED35460BDE8F0814161704701617047B0
:1013600001460548006880B200EBC100001D034A39
:1013700032F8100080B27047505C004000600040BE
:1013800001460648006880B200EBC100801D044A97
:1013900032F81000C0F3090070470000505C0040B4
:1013A0000060004001460548006880B200EBC100C3
:1013B000034A32F8100080B270470000505C0040D1
:1013C00000600040014629B90120034A12681082DA
:1013D000002070470148FCE7E403002040030020A0
:1013E00070B50A480468001D0568001D066834448D
:1013F00054B108220649204600F056F80422044958
:101400001031284600F050F870BD0000E8F7FF1FCB
:10141000EA02002070B50548446825460449086082
:1014200001460868FEF797FEA84770BD0000010856
:1014300008ED00E000BFFEE710B518480068047A28
:10144000022C01D0042C05D1FFF72EFC13480068B4
:10145000047A1CE0062C19D1104800684078052851
:101460000ED10E480068007800F07F0040B90B49AB
:101470000968C87800F046FF09490968086A80478A
:101480000849096888688047082400E0082403495F
:1014900009680C7200F09EFB10BD0000E403002000
:1014A000F0030020E803002030B50B46002100BF08
:1014B00016E00A24B4EB107F05D9302404EB107435
:1014C00003F8114005E0412404EB10740A3C03F8D2
:1014D0001140000100254C00641C1D554C1CE1B25C
:1014E0009142E6DB30BD704710B54FF480410248B1
:1014F000FFF732FF10BD00000018014010B54FF497
:1015000080410248FFF72AFF10BD0000001801408B
:1015100010B5002000F018F810BD0000014659B9C0
:101520004FF48060054A10604010054A1060800248
:10153000044A1060002070470120FCE730020020C0
:10154000280200202002002010B5044614B1012C0E
:1015500005D102E002F0AAFE03E0012010BD012047
:10156000FCE700BF0020F9E72DE9F04106460F46F1
:1015700014461D4616B1012E12D110E00CE04FF4B6
:1015800080723946204602F009FFA5F5807085B2C9
:1015900007F5807704F58074002DF0D103E002E0B8
:1015A0000120BDE8F08100BF0020FAE72DE9F041FD
:1015B00007460C4615461E4617B1012F10D10EE006
:1015C0000AE02946204602F05FFFA6F5807086B249
:1015D00004F5807405F58075002EF2D103E002E079
:1015E0000120BDE8F08100BF0020FAE770B5054694
:1015F000002414480068007800F07F00212810D1F2
:10160000FE2D0ED10F480068408850B90D48006883
:10161000808830B90B480068C088012801D10A4C85
:1016200001E0022070BD0CB90220FBE7054800680C
:10163000846100210348006841820020A047002007
:10164000F0E70000E4030020C513000810B50446CD
:101650000249204601F014F910BD0000A403002047
:1016600010B504460249204601F00AF910BD0000F9
:101670009C03002070B5054606480068C478052C18
:1016800001DD002070BD044800EBC401284601F0D4
:10169000F7F8F7E7E4030020AC0300200246002936
:1016A00001DD02207047002A01DD0220FAE7002058
:1016B000F8E7000010B5044611480068007800F013
:1016C0007F0021281AD1FF2C18D10D4800684088CE
:1016D000A0B90B480068808880B909480068C088B4
:1016E00060B90120FFF7F8F80220FFF7DBF80548A2
:1016F0000549086000200549087010BD0220FCE77C
:10170000E4030020555342439C110020DC020020DA
:1017100010B50020324988723248C07932490968D0
:101720004872002000F0E6FD4FF40071002000F048
:10173000C1FE2021002000F09DFE1821002000F0B5
:1017400009FE2A4890F82C10002000F015FE5821C0
:10175000002000F071FE0020FFF7D8F8002000F014
:1017600051FE0021012000F0A5FE9821012000F08B
:1017700063FE2021012000F07DFE0021012000F009
:1017800021FE0021022000F095FED821022000F069
:10179000E1FD164890F82C10022000F0EDFD4FF40A
:1017A0004051022000F00EFE0021022000F062FEF7
:1017B0000E4890F82C10002000F0DEFD002000F014
:1017C00021FE002000F09EFD012009490860094823
:1017D0000949086000200949087001F0B5FA10BDF8
:1017E000CC11002084450008E403002048030020B9
:1017F000D4030020555342439C110020DC020020FA
:101800007047704710B5FFF7EBFD002005490968E8
:10181000887200F003FA01F099FA0020024908608A
:1018200010BD0000E4030020D403002010B50448DC
:1018300000680449884202D00220FEF700FD10BD76
:101840009C1100205553424310B5184800780228D7
:1018500010D003281DD0042802D0052823D100E091
:1018600000BF0020114908704FF44051022000F0E1
:10187000A9FD19E00E48C07B282808D10C49487BF7
:101880000C490A680C49096800F06CFB00BF00BFF6
:101890000AE00121002000F093FE4FF440510220A5
:1018A00000F090FD00E000BF00BF10BDDC02002092
:1018B0009C110020E4020020E002002010B51D4829
:1018C000C47B1D49022001F053FA1C4908801C48C2
:1018D000007810B101281CD102E0FEF7D9FC26E007
:1018E0002A2C08D11349487B16490A681649096809
:1018F00000F05EFC1BE00120FEF7A1FC0D49487BD7
:101900002422052100F07AFE0021022000F058FE7A
:101910000DE00220FEF793FC0649487B24220521B6
:1019200000F06CFE0021022000F04AFE00BF00BF64
:1019300010BD00009C1100205C110020DE02002080
:10194000DC020020E4020020E002002010B508487C
:101950000068807A58B10520064908600120FEF72A
:10196000BBFF0220FEF79EFF00200349087010BD58
:10197000E4030020D4030020DC02002004200149FD
:1019800008607047D403002000BFFEE7704770472F
:1019900070B5002100230F22C47804B3154C2468CD
:1019A00004F4E064C4F5E064210AC1F10403CA4010
:1019B000447804FA03F184781440214309010E4C61
:1019C0000678A155047804F01F050124AC40057881
:1019D0006D11AD0005F1E025C5F8004109E004787E
:1019E00004F01F050124AC40044D0678761145F83B
:1019F000264070BD0CED00E000E400E080E100E076
:101A000002490143024A1160704700000000FA05D4
:101A10000CED00E070B502264A4800684478494859
:101A20000068007800F07F0000284AD1092C03D11B
:101A300000F0CEFF064665E0052C14D14148006851
:101A4000C0787F280BDC3F480068807838B93D4873
:101A50000068808818B93B480068807A08B108257A
:101A60006BE000264EE0032C14D136480068C078A5
:101A700001280DD133480068808848B93148006892
:101A8000407A00F0200018B100F0C6FF064639E0A9
:101A9000022637E0012C35D12A480068C078012899
:101AA0000DD128480068808848B926480068407AE7
:101AB00000F0200018B100F017FE064622E00226D2
:101AC00020E020480068007800F07F00012805D160
:101AD0000B2C17D101F01CF8064613E019480068DA
:101AE000007800F07F0002280BD1012C03D100F018
:101AF000FBFD064606E0032C04D100F0A1FF0646DC
:101B000000E002264EB1E0B20F4A126851698847E0
:101B10000646032E01D109250FE00EB108250CE081
:101B2000062500210948006880B2801C084A42F856
:101B3000101030200749088000BF024909680D7263
:101B400070BD0000E4030020E8030020505C00406A
:101B500000600040F603002010B511480068047AC8
:101B6000022C01D0042C01D1082412E0032C01D056
:101B7000052C05D1FFF7F8F809480068047A08E059
:101B8000072C05D107490968C8688047082400E088
:101B90000824034909680C7200F01CF810BD00000D
:101BA000E4030020E8030020F0B5561C7510074E32
:101BB00006EB41042B4605E034F8047B20F8017B5A
:101BC000401C5B1E002BF7D1F0BD00000060004000
:101BD0007047000010B50D4890F82C10002000F060
:101BE000CBFB0B480068007A082805D14002094960
:101BF000088010200849088005480068007A0928F4
:101C000001D1012010BD0020FCE7000048030020A6
:101C1000E4030020F4030020F603002010B50120A7
:101C200000F0FAFF01240B48046000200A490880F4
:101C300008460088074908600020091D08604FF425
:101C4000E0500549088008460088024908600020E5
:101C500010BD0000405C0040EE03002029B1064AA0
:101C6000D2690243044BDA6104E0034AD269824339
:101C7000014BDA61704700000010024029B1064AAA
:101C800012690243044B1A6104E0034A1269824359
:101C9000014B1A61704700000010024029B1064A4A
:101CA00092690243044B9A6104E0034A92698243B9
:101CB000014B9A61704700000010024029B1064AAA
:101CC000D2680243044BDA6004E0034AD2688243DC
:101CD000014BDA60704700000010024001490860C3
:101CE00070470000D800424270B504460D461646C3
:101CF0003748007870B9374850F8240068433649AF
:101D00000860344850F824007043344908600120CA
:101D10002F4908702E480078012846D130480068C5
:101D2000C0B92C4830F8240083B22E4A2A480168F2
:101D30002046FFF719FC40222A49812001F02FF8A4
:101D4000244850F82400403825490860402026499E
:101D5000086011E02348244A12688118402281203B
:101D600001F01DF81E48006840381D4908601E48F3
:101D7000006840301C4908604021012000F06CFBE5
:101D80003021012000F076FB1348006840301249F2
:101D9000086012480068403810490860134880689D
:101DA000403812498860FFF7A9FB0C48006870B9F9
:101DB00000200B4908600C490860074908600320AF
:101DC0000B490870002002490870FFF78DFB70BDB9
:101DD00048020020280200204C020020500200206F
:101DE000380200205C0900203C020020BC110020C9
:101DF000DC0200202DE9F04104460D4617461E4640
:101E0000B8191C4951F82410884213D92A2D02D13F
:101E10000220FEF714FA0020FEF711FA2122052114
:101E2000204600F0EBFB0021012000F0C9FB002060
:101E3000BDE8F08110488168104850F824007043D4
:101E4000814214D02A2D03D10220FEF7F8F902E0D6
:101E50000020FEF7F4F90849487B2422052100F010
:101E6000CDFB0021012000F0ABFB0020E0E70120CA
:101E7000DEE70000300200209C1100202802002034
:101E800010B504462046FFF749FB68B10749487B77
:101E90003A22022100F0B2FB0121084600F090FB3B
:101EA0000020FEF7CCF910BD00BFFCE79C1100201C
:101EB00070B506460C48007C00F0010010B10B4CD8
:101EC0002A250BE00EB90A4C00E00A4C0648C07CFB
:101ED000242802DC0448C57C00E02425294620464D
:101EE00000F07EFE70BD00009C1100205C0200200E
:101EF000610200208402002010B504460E4880686C
:101F000018B90020FEF79BF90BE00B48007B00F0AE
:101F1000800018B10020FEF792F902E00220FEF7DF
:101F20008EF90549487B2022052100F067FB00213E
:101F3000012000F045FB10BD9C11002010B50446A7
:101F40000821024800F04CFE10BD0000AC02002049
:101F500010B504460421024800F042FE10BD000006
:101F6000A802002070B506460C46154619480078B0
:101F700020BB1949487B2B4622462821FFF73AFF10
:101F800000B970BD1448007B00F0800040B1022011
:101F9000104908702A4621463046FFF7A5FE0CE09E
:101FA0000220FEF74CF90C49487B2422052100F061
:101FB00025FB0121084600F003FBE2E70548007815
:101FC000022804D12A4621463046FFF78DFE00BF85
:101FD000D7E70000DC0200209C11002010B5044669
:101FE0002046FFF79BFA68B11F49487B3A2202213D
:101FF00000F004FB0121084600F0E2FA0020FEF7A1
:102000001EF910BD194850F82400401E000E184952
:102010000870164850F82400401E000C4870134801
:1020200030F82400401E000A8870104810F8240080
:10203000401EC8700F4850F82400000E08710D486B
:1020400050F82400000C48710A4830F82400000AB7
:102050008871084810F82400C8710821044800F06D
:10206000BFFD00BFCDE700009C1100203002002022
:10207000C60200202802002010B504462046FFF7C3
:102080004DFA68B11A49487B3A22022100F0B6FAAB
:102090000121084600F094FA0020FEF7D0F810BDA8
:1020A000144850F82400000E13490871114850F8E4
:1020B0002400000C48710F4830F82400000A887191
:1020C0000C4810F82400C8710C4850F82400000C8B
:1020D00048720A4830F82400000A8872074810F84D
:1020E0002400C8720C21044800F07AFD00BFD6E736
:1020F0009C11002030020020CE0200202802002087
:1021000070B505460648C07C122802DC0448C47C31
:1021100000E012242146034800F062FD70BD00007B
:102120009C110020B402002010B5044601210020BB
:1021300000F046FA10BD000010B504462046FFF737
:10214000EDF968B10949487B3A22022100F056FABC
:102150000121084600F034FA0020FEF770F810BDA7
:102160000121002000F02CFA00BFF8E79C110020AC
:1021700010B504460D48806848B90C48007C00F052
:10218000040020B90121002000F01AFA0CE002201E
:10219000FEF755F80549487B2422052100F02EFA68
:1021A0000021012000F00CFA10BD00009C1100205D
:1021B00070B506460C4615461948007820BB1949EB
:1021C000487B2B4622462A21FFF714FE00B970BD3A
:1021D0001448007B00F0800040B9012010490870CD
:1021E0004FF44051022000F0EDF80CE00020FEF723
:1021F00026F80C49487B2422052100F0FFF9002134
:10220000012000F0DDF9E2E705480078012804D15B
:102210002A462146304600F0F7FD00BFD7E7000010
:10222000DC0200209C11002021B1028842F0400213
:10223000028004E002884FF6BF731A4002807047A4
:1022400010B504461148844208D101218014FFF7DB
:1022500035FD0021A014FFF731FD16E00C48844243
:1022600008D101210014FFF709FD00212014FFF718
:1022700005FD0AE00748844207D10121C013FFF79A
:10228000FDFC0021E013FFF7F9FC10BD0030014018
:1022900000380040003C00400246002013890B40FB
:1022A0000BB1012000E0002070470146888970478B
:1022B0008181704710B50022028802F441520B88D8
:1022C0004C8823438C882343CC8823430C892343A5
:1022D0004C8923438C892343CC8923431A430280AE
:1022E000838B4FF2FF74234083830B8A038210BDDC
:1022F000704700004FF6F8710140014A11607047C5
:10230000505C004030B501460F4B1A78002014E0B5
:1023100003060E4C04EB9353D3F8003C48F68F743D
:10232000234048F280042343C4B223430406074DEC
:1023300005EB9454C4F8003C401C9042E8D341F0B3
:102340008003034C236030BD440300200050004054
:102350004C5C004010B54A105300054A126892B216
:1023600002EBC002121D034C44F8123010BD0000F5
:10237000505C00400060004010B502460F48006805
:1023800080B200EBC200801D0D4C04EB40033E29DF
:102390000BDD481101F01F040CB9441EA0B24FF42C
:1023A000004444EA80241C6007E0481001F0010466
:1023B0000CB1441CA0B284021C6010BD505C0040F3
:1023C0000060004030B50E4C04EB8003D3F8003CB5
:1023D0004BF68F7403EA040201F480530BB182F4CC
:1023E000805201F400530BB182F4005242F40043D6
:1023F00043F08003024D05EB8004C4F8003C30BD7F
:102400000050004010B50B4B03EB8002D2F8002CBB
:102410004BF68F7302EA030181F4805181F400517D
:1024200041F4004242F08002024C04EB8003C3F806
:10243000002C10BD0050004010B54A105200044B53
:102440001B689BB203EBC003024C44F8132010BD81
:10245000505C004000600040044A126892B202EBF7
:10246000C002921C024B43F812107047505C0040AF
:102470000060004030B50E4C04EB8003D3F8003C04
:1024800048F6BF7403EA040201F010030BB182F0B6
:10249000100201F020030BB182F0200242F400434D
:1024A00043F08003024D05EB8004C4F8003C30BDCE
:1024B0000050004010B5074B03EB8002D2F8002C0F
:1024C00048F68F131A400A43024C04EB8003C3F80A
:1024D000002C10BD0050004010B500F001F810BDF8
:1024E0000CB50020019000903348006840F4803023
:1024F0003149086000BF3048006800F400300090A7
:102500000198401C0190009818B90198B0F5A06F8F
:10251000F1D12948006800F4003010B1012000908A
:1025200001E0002000900098012843D12348006872
:1025300040F01000214908600846006820F00300C0
:1025400008600846006840F0020008601A484068C9
:10255000194948600846406848600846406840F4A9
:10256000806048600846406820F47C104860084657
:10257000406840F4E81048600846006840F0807009
:10258000086000BF0C48006800F000700028F9D017
:102590000948406820F00300074948600846406841
:1025A00040F00200486000BF0348406800F00C00A3
:1025B0000828F9D10CBD00000010024000200240A4
:1025C00070B505460C460A480A4908600846057376
:1025D0000D22812000F0E3FB0520074908702CB193
:1025E0000420087030210120FFF744FF70BD000077
:1025F00055534253BC110020DC020020014B99705E
:102600001A737047B402002010B500F0B9FA00F058
:1026100015FBFEF768FFFEF77BFF10BD10B500202D
:10262000FFF75CFB0121C805FFF718FB10BD000098
:1026300038B501242948006880B2001D284931F8C6
:10264000100080B201EB4000009026480068007A3C
:10265000092832D00098007822490968087000984B
:10266000401C0090009800781E4909684870009846
:10267000401C0090009800EB44000090009931F855
:10268000020B0091FDF7FDFD16490968488000988E
:1026900000EB44000090009931F8020B0091FDF727
:1026A000F0FD104909688880009800EB4400009014
:1026B000009800880B490968C88001200949096809
:1026C000087208480068C08810B9FFF7A3F901E054
:1026D000FEF7A8FBFFF77EFA38BD0000505C004013
:1026E00000600040E40300202DE9F04754480068F2
:1026F000007800F07F08B8F1000F0AD15048006858
:10270000407A00F0DF004E49096848720020BDE8B9
:10271000F087B8F1020F7CD149480068408818B9A9
:1027200047480068007908B10220F0E7DFF814910B
:1027300043480068477927F080052C4640480068E8
:10274000407900F0800038B13F4901EB8400D0F8B7
:10275000000C00F0300606E03B4901EB8400D0F8A5
:10276000000C00F4405699F80000A84204D91EB1AC
:1027700033480068807A08B90220C8E707F0800073
:1027800080B1314901EB8400D0F8000C00F030003A
:1027900010284BD1E0B2FEF79FF8E0B23021FFF7EE
:1027A00069FE43E0284901EB8400D0F8000C00F4F6
:1027B0004050B0F5805F39D1E4B9244A92F82C102A
:1027C000E0B2FFF7D9FD204A02EB8401D1F8001CEA
:1027D0004BF68F7201EA020080F4805080F40050C2
:1027E00040F4004141F08001174B03EB8402C2F832
:1027F000001C1BE0E0B2FEF755F8134A02EB84011F
:10280000D1F8001C4BF68F7201EA020080F4805070
:1028100000E011E080F4005040F4004141F08001FC
:10282000094B03EB8402C2F8001C00BF0849096889
:102830004869804700206AE700BF022067E7000080
:10284000E40300204403002000500040480300201F
:10285000F003002010B504462CB901200649096890
:102860000882002010BD05490968086880470248B1
:1028700000680A30F6E70000E4030020F0030020BF
:1028800010B5024606480068438A32B98888C01AE3
:10289000034C24682082002010BD08681844FBE720
:1028A000E403002010B504462CB90120064909684C
:1028B0000882002010BD05490968886880470248E1
:1028C00000680C30F6E70000E4030020F00300206D
:1028D00010B504462CB90220394909680882002045
:1028E00010BD00203749088035480068007800F0A6
:1028F0007F0018BB32490968487A00F0200131B1E5
:102900003049097841F002012E4A117005E02D4945
:10291000097801F0FD012B4A117000F0400131B13E
:102920002849097841F00101264A117005E025493E
:10293000097801F0FE01234A11703AE0204800684E
:10294000007800F07F00012801D11E48C8E71C482C
:102950000068007800F07F00022828D1184A126829
:10296000517901F00F0001F080027AB1164B03EBB0
:102970008002D2F8002C02F03002102A16D1114A3F
:10298000127842F001020F4B1A700FE00E4B03EB6E
:102990008002D2F8002C02F44052B2F5805F05D1DB
:1029A000084A127842F00102064B1A7001E000203A
:1029B00096E70649096808698047024890E70000E1
:1029C000E4030020DC03002000500040F00300205E
:1029D00010B50E480068C0780D494978884213DC6C
:1029E0000A480068807878B908480068808858B933
:1029F00006480068C0780549096888720549096871
:102A000048688047002010BD0220FCE7E403002056
:102A100044030020F003002010B507480068407A06
:102A200040F0200004490968487204490968C869EF
:102A30008047002010BD0000E4030020F0030020C8
:102A40002DE9F0412E480068467926F080073C4683
:102A50002B480068407900F0800038B1294901EB2B
:102A60008400D0F8000C00F0300506E0254901EBA9
:102A70008400D0F8000C00F4405523480078A042B0
:102A800008D91F480068408820B91DB11C4800685B
:102A9000807A10B90220BDE8F08106F08000A0B174
:102AA000184A02EB8401D1F8001C48F6BF7201EA13
:102AB000020080F0100040F4004141F08001114B11
:102AC00003EB8402C2F8001C14E00E4A02EB8401FE
:102AD000D1F8001C4BF68F7201EA020080F480509E
:102AE00040F4004141F08001064B03EB8402C2F840
:102AF000001C00BF05490968886980470020CAE7B3
:102B0000E40300200050004044030020F0030020B4
:102B100010B5174B1B68D978154B1B685879154BA6
:102B20001B689A699047044611480068807AE8B1AA
:102B30003CB90F480068007918B90D4800688078E2
:102B400008B1022010BD8CB90B490968C8688047DC
:102B500007480068407906490968C8720448006857
:102B6000C0780349096808730020EBE70220E9E711
:102B7000E4030020E8030020F00300207047000079
:102B800010B51348006840F001001149086008467C
:102B90004068104908400E494860084600680E49E0
:102BA00008400B4908600846006820F4802008604F
:102BB0000846406820F4FE0048604FF41F0088601B
:102BC000FFF78AFC4FF000600449086010BD000068
:102BD000001002400000FFF8FFFFF6FE08ED00E0E5
:102BE00070B505460C4622462946812000F0D7F8EC
:102BF00030210120FFF73EFC0320054908700548FD
:102C00008068001B034988600020087370BD0000C5
:102C1000DC020020BC11002010B504462CB14FF49A
:102C200080410548FEF79AFB04E04FF480410248DA
:102C3000FEF792FB10BD00000018014008B501210D
:102C40000420FFF72BF84FF48060ADF8000003205C
:102C50008DF8020014208DF8030069460148FEF744
:102C6000F0FA08BD0008014010B5FDF773FC10BD77
:102C700010B508480849086002200968087207482A
:102C80000749086007480849086005490968086855
:102C9000804710BDCC110020E40300204803002031
:102CA000E803002078030020F003002008B54FF46B
:102CB000C060FEF7A5FE14208DF8000001208DF8FD
:102CC00001008DF802008DF803006846FEF760FEF3
:102CD00013208DF8000001208DF8010000208DF8F0
:102CE000020001208DF803006846FEF751FE08BD82
:102CF00010B50F4800680F4908800846008800F4A6
:102D000000400D490988084008B1FDF787FC0948D3
:102D1000008800F4806008490988084030B14FF607
:102D2000FF300349086005494868804710BD00002E
:102D3000445C004004030020EE0300204803002010
:102D400010B5FFF7D5FF10BD704700000020064901
:102D500008604FF40440054908800846008802498D
:102D6000091F086000207047445C0040EE0300200B
:102D70002DE9F04104460E46002504F07F00FEF7E1
:102D8000FFFA054604F07F00FEF7EAFA07462A46F6
:102D900039463046FEF708FF2846BDE8F0812DE9A8
:102DA000F04104460E46154604F07F00FEF7FAFA9D
:102DB0000746AAB23946304600F00AF8A9B204F034
:102DC0007F00FFF749FB0020BDE8F08100BFFEE770
:102DD000F0B5144604F1010C4FEA6C07DFF824C08B
:102DE0000CEB41033D460AE00678401C90F800C019
:102DF00046EA0C2223F8022B9B1C401C6D1E002D62
:102E0000F2D1F0BD006000402DE9F04104460D46CE
:102E100016463E48006800F140073D48007870B90A
:102E20003C4850F8240068433B490860394850F852
:102E3000240070433949086001203549087034483E
:102E4000007801284ED100203549086010E0344850
:102E500001680068401C324A10603248415C3248C8
:102E60002A4A1268815429480068401C2749086092
:102E700026480068B842EAD3274800682B490988E9
:102E80000844254908602548006828490988401AEF
:102E9000224908601F4850F824000968B1FBF0F28D
:102EA00000FB121080B9002018490860194830F85A
:102EB000240083B2174850F82400174A1268111AE8
:102EC000194A2046FEF772FB19488068174909889D
:102ED000401A174988604FF440510220FFF772FAF8
:102EE000FEF70CFB0D48006818B112480078042862
:102EF0000AD10020054908600121FFF761FB00208D
:102F000003490870FEF7F0FABDE8F08140020020A6
:102F1000480200202802002054020020580200200D
:102F2000440200205C1100205C090020DE02002029
:102F3000BC110020DC0200200FB4084B10B504A91E
:102F400002AA039800F01CF8044602A9002000F031
:102F5000B8F9204610BC5DF814FB0000C33200082D
:102F600002E008C8121F08C1002AFAD17047704752
:102F7000002001E001C1121F002AFBD170470000B0
:102F80002DE9FF4F8BB088460546002606E0252830
:102F90000BD0DDE90D1290476D1C761C28780028B7
:102FA000F5D10FB03046BDE8F08F0024A146A2460F
:102FB0000122AE4900E0044315F8013F203B02FA2C
:102FC00003F00842F7D128782A2810D06FF02F029A
:102FD0002878A0F13001092915D809EB890102EB05
:102FE000410144F0020400EB01096D1CF0E758F8C0
:102FF000041B5FEA010903D544F40054C9F1000938
:1030000044F002046D1C28782E2817D115F8010F02
:1030100044F004042A280ED06FF02F022878A0F183
:10302000300109290AD80AEB8A0102EB410100EBC1
:10303000010A6D1CF2E758F804AB6D1C28786C2867
:103040000FD006DC4C2817D068280DD06A2814D180
:1030500004E0742810D07A280FD10DE044F4001455
:103060000AE044F4801401E044F440146978814299
:1030700002D104F580146D1C6D1C2878692865D078
:1030800006DC00288DD0632827D0642806D15DE0B7
:103090006E2808D073282AD0752877D0DDE90D1264
:1030A0009047761CE0E0C4F30250022809D00328C0
:1030B0000DD0D8F8001004280DD00E6008F10408D7
:1030C000D2E0D8F80010F217C1E90062F6E7D8F8AC
:1030D00000100E80F2E70E70F0E718F8041B8DF870
:1030E000001000208DF80100EB46012003E058F8A5
:1030F00004BB4FF0FF3061074FF0000701D40AE036
:103100007F1C57450DDA8742FADB1BF807100029B0
:10311000F6D106E07F1C8742FCDB1BF80710002974
:10312000F8D1DDE90D23A9EB07008146214600F027
:10313000B1F83044C61904E0DDE90D121BF8010BAB
:1031400090477F1EF8D22146484688E058F8040B85
:10315000C4F302514FF00A0B032900D100B2042935
:1031600000D140B2002802DA40422D2102E02105C0
:1031700005D52B218DF82410012104E006E0E1079C
:1031800010D02021F6E708AF089113E058F8040B9F
:10319000C4F302514FF00A0B032900D180B2042975
:1031A00000D1C0B20021EEE75946FCF7F4FF303100
:1031B00007F8011D0028F7D1ADEB070000F1200B47
:1031C000600702D524F4803401E04FF0010ADA45AB
:1031D00002DDAAEB0B0000E00020824600EB0B01B1
:1031E00008980144A9EB01000A90E00306D4DDE948
:1031F0000D2321460A9800F04DF806444FF00009CF
:1032000008E009A911F80900DDE90D12904709F15C
:103210000109761C08998945F3DBE0030CD5DDE94B
:103220000D2321460A9800F035F8064404E0DDE954
:103230000D1230209047761CBAF10001AAF1010A64
:10324000F5DC05E0DDE90D1217F8010B9047761C5F
:10325000BBF10001ABF1010BF4DC0A982146DDE97A
:103260000D2300F005F806446D1C97E609280100BF
:103270002DE9F041044600251E461746880404D473
:1032800005E039462020B0476D1C641EF9D528465C
:10329000BDE8F0812DE9F041044600251E46904628
:1032A000C80301D5302700E02027880404D505E0B5
:1032B00041463846B0476D1C641EF9D52846BDE826
:1032C000F0810A68531C0B601070704770B504469B
:1032D0000D46002084F80402401EC4F8240229464A
:1032E000204600F0CBFF08B1032070BD94F8FE111A
:1032F00040F2FF10005D41EA00204AF65521884265
:1033000001D00220F1E73920005D01063820005D80
:1033100041EA00413720005D41EA002094F8361070
:10332000084320F07F400E49884201D10020DCE7AD
:103330005520005D01065420005D41EA0041532004
:10334000005D41EA002094F85210084320F07F40CD
:103350000349884201D10020C7E70120C5E70000EA
:1033600046415400024600E0521C107810B110781B
:103370008842F9D1107870470246891ED2F80C02B3
:10338000801E884201D80020704792F80232D2F89D
:10339000200201FB0300F7E72DE9F35F8A46DAF824
:1033A000007000E07F1C38782F28FBD038785C282C
:1033B000F8D00098D0F818620B222021304600F097
:1033C00053FF0025A946AB464FF0080800BF5846FA
:1033D0000BF1010B3C5C202C03DD2F2C01D05C2C6D
:1033E00000D134E02E2C01D0C1450ED3B8F1080F26
:1033F00001D12E2C02D00620BDE8FC9F4FF0080919
:103400004FF00B08A806050EE1E7802C03DB45F022
:1034100003050620F0E7214621A0FFF7A3FF08B12E
:103420000620E9E7412C04DB5A2C02DC45F00205BA
:1034300008E0612C06DB7A2C04DC45F00105A4F1E0
:103440002000C4B2484609F101093454BFE700BF67
:1034500007EB0B00CAF80000202C01DC042000E080
:1034600000200446B9F1000F01D10620C4E73078EE
:10347000E52801D105203070B8F1080F01D1A80668
:10348000050E05F00300012801D144F0100405F0F9
:103490000C00042801D144F00804F4720020ABE7CA
:1034A000222A2B2C3A3B3C3D3E3F5B5D7C7F00005B
:1034B0002DE9F04104460021204600F085F805463C
:1034C00015B12846BDE8F08100BFD4F81012D4F839
:1034D000000200F0D3FE054605B118E0D4F81462EE
:1034E00037780FB9042512E0F07A00F0080038B9F7
:1034F0000B223046D4F8181200F096FE00B906E010
:103500000021204600F006F80546002DDDD000BF62
:103510002846D7E72DE9F04104460F46B4F80602E5
:10352000461CB0B210B1D4F8100210B90420BDE8A6
:10353000F08106F00F0078BBD4F81002401CC4F8EC
:103540001002D4F80C0238B9D4F80002B0F808021E
:10355000B0422DD80420EAE7D4F8000290F8020225
:10356000401E00EA1610B8B9D4F80C12D4F80002C4
:1035700000F080FC0546012D01D80220D7E7681C29
:1035800008B90120D3E7D4F80002D0F80C02A84211
:1035900005D817B90420CAE70AE00420C7E7C4F831
:1035A0000C522946D4F80002FFF7E6FEC4F81002D8
:1035B000A4F8066206F00F00D4F8001201EB4010E8
:1035C000C4F814020020B2E72DE9F04104460E468B
:1035D000A4F80662D4F80852012D05D0D4F80002F0
:1035E000D0F80C02A84202D80220BDE8F0814DB903
:1035F000D4F8000290F80002032803D1D4F80002A6
:10360000D0F81C5265B9D4F80002B0F80802B042F4
:1036100001D80220E9E7D4F80002D0F81C7224E0B7
:10362000D4F8000290F802024FEA001815E029468B
:10363000D4F8000200F01EFC0546681C08B9012001
:10364000D3E7022D05D3D4F80002D0F80C02A8422B
:1036500001D80220C9E7A6EB08064645E7D229466D
:10366000D4F80002FFF788FE0746C4F80C520FB9E1
:103670000220BAE707EB1610C4F8100206F00F009C
:10368000D4F8001201EB4010C4F814020020ACE79B
:1036900001460020704700002DE9F04107460D4625
:1036A00014461E467600640011E021024FF4807239
:1036B000284600F073FE084928680968884202D14C
:1036C000200206490860641C05F58075761E002EF0
:1036D000EBD10020BDE8F081200000201C0000207C
:1036E00001460020704770B50446204600F00CFFEC
:1036F000054615B90020C4F80002284670BD2DE922
:10370000F04704460D46204600F0FEFE8246BAF120
:10371000000F02D05046BDE8F08794F8070210B1C0
:1037200094F80702F7E7D4F80C02A84201D2D4F8C3
:103730000C52D4F808924FF00008C4F80882002D0B
:103740005CD0D4F8000290F802024702B9F1000FF1
:1037500014D0681EB0FBF7F1A9F10100B0FBF7F03F
:1037600081420BD3A9F10100791E8843C4F80802F5
:10377000D4F808022D1AD4F8146203E0D4F81062C9
:10378000C4F81462BEB31FE03146D4F8000200F062
:1037900071FB0646701C18B9012084F80702BAE7CD
:1037A000012E05D9D4F80002D0F80C02B04203D89B
:1037B000022084F80702AEE7C4F81462D4F80802C5
:1037C0003844C4F80802ED1BBD42DDD8D4F8080225
:1037D0002844C4F80802C5F3080060B13146D4F8A3
:1037E0000002FFF7C9FD8046B8F1000F04D10220A6
:1037F00084F807028FE701E008EB5528B4F80802C7
:10380000C0F3080098B1D4F8180240450FD0D4F89E
:10381000001291F80102012342462146FFF73CFFC6
:1038200018B1012084F8070275E7C4F818825046E1
:1038300071E70000F7B582B016460398019001A821
:1038400000F0C8FB0546002D02DA0B2005B0F0BDE4
:103850000F4850F8254014B1002084F80002029867
:1038600018B10020029981F800020949029841F834
:103870002500029808B1012E01D00020E6E70022C1
:1038800003A902A800F03CF907463846DEE700002D
:10389000F8030020F7B5ADF50A7D044617461CB9BC
:1038A00009200DF50D7DF0BD0020C4F8000207F0E1
:1038B000010700228BA983A800F022F90646002EFA
:1038C00032D1CDF824D203A88B9900F085FA0646B0
:1038D000889D46B9889D0DB9062604E0E87A00F077
:1038E000100000B10426FEB904F50074A771002091
:1038F000E0712946839800F091FB2061E87F010682
:10390000A87F41EA0041687F41EA0020297F0843FF
:10391000E0600020A060A061839820602068B0F87B
:103920000602A080A4F500743046BAE72DE9FF4FE7
:1039300083B0044615469946049800900020C9F8C3
:103940000000204600F0E0FD0290029818B10298B5
:1039500007B0BDE8F08F94F8070210B194F80702A1
:10396000F6E794F8060200F0010008B90720EFE737
:10397000D4F80812D4F80C02401A0190019885423C
:1039800000D9019D96E0B4F80802C0F308000028B1
:103990006FD1D4F8000290F80202401ED4F8081249
:1039A00000EA512000F0FF08B8F1000F1CD1D4F854
:1039B000080210B9D4F810B206E0D4F81412D4F802
:1039C000000200F057FA8346BBF1020F03D2022037
:1039D00084F80702BCE70BF1010018B9012084F854
:1039E0000702B5E7C4F814B2D4F81412D4F80002F0
:1039F000FFF7C2FC07461FB9022084F80702A7E7B9
:103A000047444FEA552ABAF1000F1ED008EB0A00CE
:103A1000D4F8001291F80212884205D9D4F80002B5
:103A200090F80202A0EB080AD4F8001291F8010203
:103A300053463A460099FFF72FFE18B1012084F84B
:103A4000070285E74FEA4A2626E0D4F81802B84272
:103A50000DD0D4F8001291F8010201233A46214614
:103A6000FFF71AFE18B1012084F8070270E7C4F8C6
:103A70001872B4F80802C0F30800C0F50076AE4230
:103A800000D92E46B4F80802C0F3080001193246E6
:103A9000009800F0DCFB00BF009830440090D4F8A0
:103AA00008023044C4F80802D9F800003044C9F8CC
:103AB0000000AD1B002D7FF466AF002048E733B552
:103AC000ADF50B7D0D4600228BA984A800F018F8F7
:103AD000044684B901A88A9004A88B9900F07CF967
:103AE000044644B9899828B12DB1294604A800F0AC
:103AF00038FA00E0062420460DF50D7D30BD0000AB
:103B00002DE9F74F8AB000210A9801600B9800F068
:103B100061FA09900998002803DA0B200DB0BDE87E
:103B2000F08FAB49099851F820400CB90C20F5E70B
:103B30000A98046094F8000258B194F80102FFF763
:103B4000CFFD0890089800F0010010B900BF0020D8
:103B5000E4E7002084F80002099884F8010294F850
:103B60000102FFF795FD0890089800F0010008B1E8
:103B70000320D3E700BF4FF0000841462046FFF77F
:103B8000A5FB0546012D01D085BB2FE0002615E0E1
:103B900004F5DF7000EB0617387950B1F87A0106AA
:103BA000B87A41EA0041787A41EA0020397A08433C
:103BB00000E0002001A941F82600761C042EE7D37E
:103BC000002606B1761E00BF01A850F82680B8F185
:103BD000000F04D041462046FFF778FB00E00220AA
:103BE00005461DB1701C06460428EDD3032D01D1F6
:103BF000012093E70DB10D2090E7E17A207B41EAA7
:103C00000020B0F5007F01D00D2087E7A17DE07D89
:103C100041EA0029B9F1000F0ED12720005D01060D
:103C20002620005D41EA00412520005D41EA002098
:103C300094F8241040EA0109C4F81092207C84F81A
:103C4000030294F80302012805D094F80302022825
:103C500001D00D2062E794F8030209FB00F9607BB4
:103C600084F8020294F8020220B194F80202411E84
:103C7000084008B10D2051E7617CA07C41EA00209A
:103C8000A4F8080294F8080200F00F0008B10D2013
:103C900044E7E17C207D41EA00200790079870B955
:103CA0002320005D01062220005D41EA0041212021
:103CB000005D41EA002094F8201008430790A17BA2
:103CC000E07B41EA002BBBF1000F01D10D2025E77D
:103CD0000BEB0900B4F8081200EB11100690DDE9B7
:103CE0000601814201D20D2018E7DDE90610401AD5
:103CF00094F80212B0FBF1FABAF1000F01D10D20D5
:103D00000CE7012540F6F670824500D302254FF6F8
:103D1000F670824500D303250AF10200C4F80C02B4
:103D2000C4F8148208EB0B00C4F81802069840444B
:103D3000C4F82002032D19D1B4F8080208B10D20EF
:103D4000ECE62F20005D01062E20005D41EA0041D7
:103D50002D20005D41EA002094F82C100843C4F89F
:103D60001C02D4F80C02800005901AE0B4F8080296
:103D700008B90D20D2E6D4F818024844C4F81C0251
:103D8000022D03D1D4F80C02400009E094F80C0293
:103D900000F00100D4F80C1201EB410100EB5100DE
:103DA0000590D4F81012059800F2FF10B1EB502FD7
:103DB00001D20D20B2E684F8005206480088401C6B
:103DC00080B204490880A4F806020020A6E600009C
:103DD000F8030020FC0300202DE9F341044601987C
:103DE00000782F2803D0019800785C2802D1019830
:103DF000401C01900020C4F8080201980078202897
:103E000008D200212046FFF7DFFB05460020C4F85A
:103E100014022CE000BF01A92046FFF7BDFA0546B9
:103E200005B123E02046FFF743FB0546D4F818020E
:103E3000C67A3DB1042D04D100BF06F0040000B9DC
:103E4000052513E006F0040000B10FE0D4F8147269
:103E5000F87A00F0100008B9052507E03946D4F8D3
:103E6000000200F0DBF8C4F80802D4E700BF2846DF
:103E7000BDE8FC812DE9F04705460C46022C03D332
:103E8000D5F80C02A04202D84FF0010966E04FF0CD
:103E9000FF3995F80002012804D002282CD003280D
:103EA00058D13CE0274607EB5707D5F8180200EB3E
:103EB0005721284600F0E2F900B14EE038467F1C59
:103EC000C0F3080015F80080D5F8180200EB572160
:103ED000284600F0D3F900B13FE0C7F30800285CA2
:103EE00048EA002804F0010010B14FEA181001E080
:103EF000C8F30B00814630E0D5F8180200EB14211E
:103F0000284600F0BBF900B127E040F2FF1000EABC
:103F1000440046193078717840EA01291DE0D5F84F
:103F2000180200EBD411284600F0A8F900B114E003
:103F300040F2FF1000EA84004619F0780006B178DC
:103F400040EA0140717840EA01203178084320F0CE
:103F5000704902E04FF0010900BF00BF4846BDE8CC
:103F6000F087F0B5044601F10902D4F81062002E82
:103F70002DD0D4F81402002310E01E465B1C855D92
:103F8000202D00D10AE0052D00D1E525092B02D115
:103F90002E2602F8016B02F8015B00BF0B2BECD35D
:103FA000C67A0E72C67F3706867F47EA0647467F87
:103FB00047EA0626077F3E430E60077E467E47EAB5
:103FC00006268E80877DC67D47EA0626CE8000269F
:103FD0001670F0BD70B502464FF0FF301568DDB1C8
:103FE000116800E0491C0D78212D02D30D783A2D7F
:103FF000F8D10D783A2D0ED1146814F8015BA5F1B3
:1040000030030A2B06D28C4204D11BB918464D1C32
:104010002946156070BD002000BFFBE710B50246C1
:104020008C7ECB7E44EA032092F80032032B05D12C
:104030000C7D4B7D44EA032340EA034010BD0000A1
:104040000EB501215020FDF729FE4FF480405E4956
:104050000880032088701020C8705C48FDF7F1F8D4
:104060004FF480415948FDF779F90F2056490880EF
:104070004820C8705648FDF7E4F88020524908806F
:104080000420C8705148FDF7DCF85048083000683B
:1040900000F0800028B94F480068401C08B1FDF7C7
:1040A000B9F9FEF7B1FAFEF7B9FAFEF7FFFDFEF730
:1040B000DFFD00BF00BF45480830006800F0800009
:1040C0000028F8D1012244A14448FFF7B3FB44493A
:1040D0000870002043490860012243494348FFF724
:1040E000D9FB43490870434B4FF4807242493F4823
:1040F000FFF71CFC0020404988713C48FFF7F3FAA9
:104100003848006800284FD001223C493748FFF763
:10411000C1FB3749087008460078002844D1384967
:104120003648FFF7CCFC3648C088C0F34510344908
:10413000C988C90A324A9288520A02F2BC72CDE991
:10414000002102902E488088C0F343132C48007948
:1041500000F01F022BA13248FEF7EEFE00260024DD
:1041600017E02548005D5B2812D1002500BF2846D6
:104170006D1C2B490A5C2046641C1F49085C824266
:10418000F5D0681E2649085C212800D1012602E0EE
:10419000641CFF2CE5DD00BF36B91448D0F80C02D2
:1041A00020490860FCF7C6FB0A480068401C08B1BB
:1041B000FDF730F900BF05480830006800F08000C6
:1041C0000028F8D076E70000000000200018014029
:1041D0000010014000000108300000000004002031
:1041E000040000201C000020634500082806002071
:1041F0000500002008000020200000204A4500089B
:10420000440900205B253032752E253032752E256D
:104210007520253032753A253032752100000000B6
:10422000440800200C000020F0B503461C460D4653
:10423000002000BF1600A2F1010207D014F8017B94
:1042400015F801CBA7EB0C063000F3D0F0BD70B52C
:1042500003460C4603E014F8015B03F8015B15000C
:10426000A2F10102F7D170BD30B5034601E003F8B9
:10427000011B1400A2F10102F9D130BD70B5044652
:104280000D460026D4F82402A8420CD05EB994F85A
:10429000010201232A462146FFF7FEF908B1751EE7
:1042A0000126C4F82452304670BD000000B587B026
:1042B00001214020FDF7F2FC01210420FDF7EEFC76
:1042C00001210803FDF7EAFC4FF40060ADF804009B
:1042D00003208DF8060010208DF8070001A92C4856
:1042E000FCF7AFFF4FF400612948FDF737F8A02035
:1042F000ADF8040003208DF8060018208DF80700A3
:1043000001A92448FCF79DFFA020ADF8040003207C
:104310008DF8060018208DF8070001A91D48FCF74C
:1043200090FF4020ADF8040004208DF8070001A99B
:104330001848FCF786FF00211748FDF775FF16485F
:10434000FDF77EFF0020ADF80800ADF80C0002205C
:10435000ADF80E000120ADF810004002ADF81200DB
:104360001820ADF814000020ADF816000720ADF8B5
:1043700018004FF48270ADF80A0002A90648FDF754
:1043800099FF01210448FDF74FFF07B000BD000071
:1043900000180140000801400030014070B505469A
:1043A0000C46164600F042F84FF400611048FCF746
:1043B000D3FF032000F01EF8C4F3074000F01AF802
:1043C000C4F3072000F016F8E0B200F013F804E0A0
:1043D000A52000F00FF828706D1C3000A6F1010137
:1043E0008EB2F5D14FF400610148FCF7B7FF70BD04
:1043F0000018014010B5044600BF02210A48FDF72D
:104400004BFF0028F9D021460748FDF751FF00BFB8
:1044100001210548FDF740FF0028F9D00248FDF7CB
:1044200044FFC0B210BD00000030014010B50024B0
:104430004FF400610A48FCF78FFF0520FFF7DAFF11
:1044400000BFA520FFF7D6FF044604F001000028B6
:10445000F7D14FF400610248FCF780FF10BD000067
:104460000018014010B54FF400610648FCF774FFD6
:104470000620FFF7BFFF4FF400610248FCF76EFF14
:1044800010BD0000001801402DE9F04104460D4622
:10449000FFF7E8FF4FF400611948FCF75DFF0A20C1
:1044A000FFF7A8FFC4F30740FFF7A4FFC4F30720FA
:1044B000FFF7A0FFE0B2FFF79DFF002615E000BF69
:1044C0001048008900F002000028F9D028780D4932
:1044D000888100BF0B48008900F001000028F9D056
:1044E00008488089C7B26D1C761CFF2EE7DD4FF4AB
:1044F00000610348FCF732FFFFF798FFBDE8F08149
:10450000001801400030014070B505462C46C4B18A
:10451000D4F80002A8B1D4F8000290F8000280B1EB
:10452000D4F80002B0F80602B4F80412884208D1A8
:10453000D4F8001291F80102FFF7D2F800F0010060
:1045400008B1092070BD0020FCE72F5453343330EC
:1045500076362E62696E002F636F6E6669672E7401
:104560007874002F6C6F672E7478740076657236DD
:104570002E001201000200000040830420570002B8
:104580000102030109022000010100C032090400F8
:1045900000020806500407058102400000070502DA
:1045A000024000000403090422034E0054004B00A3
:1045B000200049006E007400650072006600610012
:1045C00063006500200031003700460354005300AB
:1045D0003400330030002000760065007200730064
:1045E00069006F006E00200036002E0030002000B1
:1045F0004E0054004B00200049006E00740065001E
:10460000720066006100630065004F004F004F00BC
:1046100010035300540020004D006100730073002C
:10462000404600080000002000040000E8010008E7
:104630001047000800040020E8110000702F000857
:1046400041031A030406FF313437370A01FF013FE3
:104650003580020220681C48592D536D61727453D5
:10466000504920466C6173684469736B2020312E79
:104670003020232D53544D20014D4E414E44243AB9
:104680002025292442036206627002150A420802AC
:104690001102141A03531254124D123312321231F2
:1046A00002113013BF100C18088F19040A15C72007
:1046B00041230301130518140811171B0801081AD8
:1046C000030413ED151408B5161B089D041A6104A4
:1046D0001A4D041A7504413240293CDA4D4C1A2D0A
:1046E00038690C1A7D041372453308121A84083293
:1046F000201AA40832041AA80832221ACA0832461C
:1047000013E80233201A1310467308101993012579
:0400000508000131BD
:00000001FF
